:020000020000FC
:0200000004C03A
:1000080076C00FED0DBF09E109B9539A23E350E01B
:10001800CC27DD2704E0502E08EE302E00E002BB8E
:1000280008BB0CEF07BB0FEF01BB09E00EBD03E0F7
:100038000BBD032D0ABD00E409BF789418C0022D3A
:10004800003412F0939A08959398089550FF0895F4
:100058005E7F022D0ED02CD0F2DF0895022D0031E4
:100068002AF4339403E00BBD032D0ABD0895EEDF97
:10007800FECF802F66277727845610F06395FCCF34
:100088008C598A5010F07395FCCF865F603039F038
:10009800605D062F12D0703011F400E30ED070307E
:1000A80019F0705D072F09D0805D082F06D00895DC
:1000B8000AE003D00DE001D008955D9BFECF509873
:1000C800529A0CB9089501E8202E5160C498C69838
:1000D800959A45990895239411F0459BFCCF08956E
:1000E800032F0F70122F107F012B08BB08950F9359
:1000F8001F938894221F08F42160062D017039F49B
:10010800032F077F302F022F06950870302BE8DF6A
:100118005A94D9F404E0502E21960C2F1D2F075E17
:10012800134090F031F4CFDF6394022D0158422C34
:10013800202E0C2F1D2F085E134011F4CC27DD272D
:100148009598949ACDDF01C094981F910F911895B6
:00000001FF
